:1000000012C02BC02AC029C028C027C026C025C0C6
:1000100024C023C022C021C020C01FC01EC01DC0DC
:100020001CC01BC01AC011241FBECFE5D4E0DEBF28
:10003000CDBF10E0A0E6B0E0ECE9F0E002C0059032
:100040000D92A036B107D9F710E0A0E6B0E001C0EC
:100050001D92A036B107E1F713C0D2CFCF93DF9343
:100060009C01892B51F0AAEFB0E0C0E0D0E0CD01B7
:100070000197F1F721503040D1F7DF91CF910895EA
:10008000CFE5D4E0DEBFCDBFA09AA89A84EF91E07F
:0C009000E5DFA89884EF91E0E1DFF7CFF6
:00000001FF
